BL51 BANKED LINKER/LOCATER V6.22                                                        05/19/2022  10:32:59  PAGE 1


BL51 BANKED LINKER/LOCATER V6.22, INVOKED BY:
C:\KEIL_V5\C51\BIN\BL51.EXE .\Objects\main.obj, .\Objects\OPTIONS_SN8F5835.obj, .\Objects\uart0.obj, .\Objects\uart1.obj
>> , .\Objects\uart2.obj TO .\Objects\UART Mode 1 PRINT (.\Listings\UART Mode 1.m51) RAMSIZE (256)


MEMORY MODEL: SMALL


INPUT MODULES INCLUDED:
  .\Objects\main.obj (MAIN)
  .\Objects\OPTIONS_SN8F5835.obj (OPTIONS_SN8F5835)
  .\Objects\uart0.obj (UART0)
  .\Objects\uart1.obj (UART1)
  .\Objects\uart2.obj (UART2)
  C:\KEIL_V5\C51\LIB\C51S.LIB (?C_STARTUP)
  C:\KEIL_V5\C51\LIB\C51S.LIB (?C?CLDPTR)
  C:\KEIL_V5\C51\LIB\C51S.LIB (?C?CSTPTR)
  C:\KEIL_V5\C51\LIB\C51S.LIB (?C_INIT)


LINK MAP OF MODULE:  .\Objects\UART Mode 1 (MAIN)


            TYPE    BASE      LENGTH    RELOCATION   SEGMENT NAME
            -----------------------------------------------------

            * * * * * * *   D A T A   M E M O R Y   * * * * * * *
            REG     0000H     0008H     ABSOLUTE     "REG BANK 0"
            DATA    0008H     0010H     UNIT         ?DT?MAIN
            DATA    0018H     000AH     UNIT         ?DT?UART0
            DATA    0022H     000AH     UNIT         ?DT?UART1
            DATA    002CH     000AH     UNIT         ?DT?UART2
            DATA    0036H     0005H     UNIT         _DATA_GROUP_
            DATA    003BH     0003H     UNIT         ?DT?_UART1_TRANSMITDATA?UART1
            IDATA   003EH     0001H     UNIT         ?STACK

            * * * * * * *  X D A T A   M E M O R Y  * * * * * * *
                    0000H     F000H                  *** GAP ***
            XDATA   F000H     0001H     ABSOLUTE     
            XDATA   F001H     0001H     ABSOLUTE     
            XDATA   F002H     0001H     ABSOLUTE     
            XDATA   F003H     0001H     ABSOLUTE     
            XDATA   F004H     0001H     ABSOLUTE     
            XDATA   F005H     0001H     ABSOLUTE     
            XDATA   F006H     0001H     ABSOLUTE     
            XDATA   F007H     0001H     ABSOLUTE     
            XDATA   F008H     0001H     ABSOLUTE     
            XDATA   F009H     0001H     ABSOLUTE     
            XDATA   F00AH     0001H     ABSOLUTE     
            XDATA   F00BH     0001H     ABSOLUTE     
            XDATA   F00CH     0001H     ABSOLUTE     
            XDATA   F00DH     0001H     ABSOLUTE     
            XDATA   F00EH     0001H     ABSOLUTE     
            XDATA   F00FH     0001H     ABSOLUTE     
            XDATA   F010H     0001H     ABSOLUTE     
            XDATA   F011H     0001H     ABSOLUTE     
            XDATA   F012H     0001H     ABSOLUTE     
            XDATA   F013H     0001H     ABSOLUTE     
BL51 BANKED LINKER/LOCATER V6.22                                                      05/19/2022  10:32:59  PAGE 2


            XDATA   F014H     0001H     ABSOLUTE     
                    F015H     0001H                  *** GAP ***
            XDATA   F016H     0001H     ABSOLUTE     
            XDATA   F017H     0001H     ABSOLUTE     
            XDATA   F018H     0001H     ABSOLUTE     
            XDATA   F019H     0001H     ABSOLUTE     
            XDATA   F01AH     0001H     ABSOLUTE     
            XDATA   F01BH     0001H     ABSOLUTE     
            XDATA   F01CH     0001H     ABSOLUTE     
            XDATA   F01DH     0001H     ABSOLUTE     
            XDATA   F01EH     0001H     ABSOLUTE     
            XDATA   F01FH     0001H     ABSOLUTE     
            XDATA   F020H     0001H     ABSOLUTE     
            XDATA   F021H     0001H     ABSOLUTE     
            XDATA   F022H     0001H     ABSOLUTE     
            XDATA   F023H     0001H     ABSOLUTE     
            XDATA   F024H     0001H     ABSOLUTE     
            XDATA   F025H     0001H     ABSOLUTE     
            XDATA   F026H     0001H     ABSOLUTE     
            XDATA   F027H     0001H     ABSOLUTE     
            XDATA   F028H     0001H     ABSOLUTE     
            XDATA   F029H     0001H     ABSOLUTE     
                    F02AH     0001H                  *** GAP ***
            XDATA   F02BH     0001H     ABSOLUTE     
            XDATA   F02CH     0001H     ABSOLUTE     
            XDATA   F02DH     0001H     ABSOLUTE     
            XDATA   F02EH     0001H     ABSOLUTE     
            XDATA   F02FH     0001H     ABSOLUTE     
            XDATA   F030H     0001H     ABSOLUTE     
            XDATA   F031H     0001H     ABSOLUTE     
            XDATA   F032H     0001H     ABSOLUTE     
            XDATA   F033H     0001H     ABSOLUTE     

            * * * * * * *   C O D E   M E M O R Y   * * * * * * *
            CODE    0000H     0003H     ABSOLUTE     
            CODE    0003H     002EH     UNIT         ?PR?_UART1_TRANSMITDATA?UART1
            CODE    0031H     0019H     UNIT         ?PR?GPIO_INITIALIZATION?MAIN
                    004AH     0009H                  *** GAP ***
            CODE    0053H     0003H     ABSOLUTE     
            CODE    0056H     000CH     UNIT         ?PR?UART0_RECEIVEDDONE?UART0
                    0062H     0001H                  *** GAP ***
            CODE    0063H     0003H     ABSOLUTE     
            CODE    0066H     0053H     UNIT         ?PR?ISR_UART0_RX?UART0
                    00B9H     000AH                  *** GAP ***
            CODE    00C3H     0003H     ABSOLUTE     
            CODE    00C6H     00ADH     UNIT         ?PR?_UART2_INIT?UART2
            CODE    0173H     00A3H     UNIT         ?PR?_UART1_INIT?UART1
            CODE    0216H     009FH     UNIT         ?PR?_UART0_INIT?UART0
            CODE    02B5H     008CH     UNIT         ?C_C51STARTUP
            CODE    0341H     0076H     UNIT         ?PR?MAIN?MAIN
            CODE    03B7H     0053H     UNIT         ?PR?ISR_UART1_RX?UART1
            CODE    040AH     0053H     UNIT         ?PR?_UART2_TRANSMITDATA?UART2
            CODE    045DH     0053H     UNIT         ?PR?ISR_UART2_RX?UART2
            CODE    04B0H     002BH     UNIT         ?PR?_UART0_TRANSMITDATA?UART0
            CODE    04DBH     002BH     UNIT         ?C?LIB_CODE
            CODE    0506H     0015H     UNIT         ?C_INITSEG
            CODE    051BH     000CH     UNIT         ?PR?UART1_RECEIVEDDONE?UART1
BL51 BANKED LINKER/LOCATER V6.22                                                      05/19/2022  10:32:59  PAGE 3


            CODE    0527H     000CH     UNIT         ?PR?UART2_RECEIVEDDONE?UART2
                    0533H     7ABDH                  *** GAP ***
            CODE    7FF0H     0002H     ABSOLUTE     
                    7FF2H     0004H                  *** GAP ***
            CODE    7FF6H     000AH     ABSOLUTE     



OVERLAY MAP OF MODULE:   .\Objects\UART Mode 1 (MAIN)


SEGMENT                                 DATA_GROUP 
  +--> CALLED SEGMENT                 START    LENGTH
-----------------------------------------------------
?C_C51STARTUP                         -----    -----
  +--> ?PR?MAIN?MAIN
  +--> ?C_INITSEG

?PR?MAIN?MAIN                         -----    -----
  +--> ?PR?GPIO_INITIALIZATION?MAIN
  +--> ?PR?_UART0_INIT?UART0
  +--> ?PR?_UART1_INIT?UART1
  +--> ?PR?_UART2_INIT?UART2
  +--> ?PR?_UART0_TRANSMITDATA?UART0
  +--> ?PR?UART1_RECEIVEDDONE?UART1
  +--> ?PR?_UART2_TRANSMITDATA?UART2

?PR?_UART0_INIT?UART0                 0036H    0005H

?PR?_UART1_INIT?UART1                 0036H    0005H

?PR?_UART2_INIT?UART2                 0036H    0005H

?PR?_UART0_TRANSMITDATA?UART0         0036H    0003H

?PR?_UART2_TRANSMITDATA?UART2         0036H    0003H



SYMBOL TABLE OF MODULE:  .\Objects\UART Mode 1 (MAIN)

  VALUE           TYPE          NAME
  ----------------------------------

  -------         MODULE        MAIN
  C:0000H         SYMBOL        _ICE_DUMMY_
  X:F003H         PUBLIC        PW1YL
  X:F017H         PUBLIC        PW2YL
  D:0080H         PUBLIC        P0
  X:F031H         PUBLIC        PW3YL
  D:0090H         PUBLIC        P1
  D:00B0H         PUBLIC        P3
  D:00C8H         PUBLIC        P4
  D:00A0H         PUBLIC        TTCON
  D:00A8H         PUBLIC        IEN0
  D:00B8H         PUBLIC        IEN1
  X:F004H         PUBLIC        PW10DH
BL51 BANKED LINKER/LOCATER V6.22                                                      05/19/2022  10:32:59  PAGE 4


  X:F018H         PUBLIC        PW20DH
  X:F006H         PUBLIC        PW11DH
  X:F01AH         PUBLIC        PW21DH
  X:F00CH         PUBLIC        PW30DH
  X:F008H         PUBLIC        PW12DH
  X:F01CH         PUBLIC        PW22DH
  X:F00EH         PUBLIC        PW31DH
  X:F00AH         PUBLIC        PW13DH
  X:F01EH         PUBLIC        PW23DH
  X:F010H         PUBLIC        PW32DH
  X:F005H         PUBLIC        PW10DL
  X:F019H         PUBLIC        PW20DL
  X:F012H         PUBLIC        PW33DH
  X:F007H         PUBLIC        PW11DL
  X:F01BH         PUBLIC        PW21DL
  X:F00DH         PUBLIC        PW30DL
  X:F009H         PUBLIC        PW12DL
  X:F01DH         PUBLIC        PW22DL
  X:F00FH         PUBLIC        PW31DL
  X:F00BH         PUBLIC        PW13DL
  X:F01FH         PUBLIC        PW23DL
  X:F011H         PUBLIC        PW32DL
  X:F013H         PUBLIC        PW33DL
  X:F000H         PUBLIC        PW1M
  C:0341H         PUBLIC        main
  X:F014H         PUBLIC        PW2M
  X:F02DH         PUBLIC        HIDR
  X:F028H         PUBLIC        P0UR
  X:F001H         PUBLIC        PW3M
  X:F029H         PUBLIC        P1UR
  X:F02BH         PUBLIC        P3UR
  X:F02CH         PUBLIC        P4UR
  D:00D8H         PUBLIC        CSCON4
  B:0080H.0       PUBLIC        P00
  B:0080H.1       PUBLIC        P01
  D:0088H         PUBLIC        TCON
  D:0008H         PUBLIC        baryUSER_RxBuf
  D:0010H         PUBLIC        baryUSER_TxBuf
  X:F027H         PUBLIC        TSWA
  X:F026H         PUBLIC        TSWB
  X:F025H         PUBLIC        TSWD
  D:00F9H         PUBLIC        P0M
  D:00FAH         PUBLIC        P1M
  D:00FBH         PUBLIC        P3M
  D:00FCH         PUBLIC        P4M
  B:00A8H.7       PUBLIC        EAL
  X:F02EH         PUBLIC        CSADB1H
  X:F024H         PUBLIC        TSWY
  X:F032H         PUBLIC        CSADB2H
  X:F02FH         PUBLIC        CSADB1L
  X:F033H         PUBLIC        CSADB2L
  C:0031H         PUBLIC        GPIO_Initialization
  D:0098H         PUBLIC        S0CON
  X:F022H         PUBLIC        MINCS0H
  X:F020H         PUBLIC        MAXCS0H
  X:F023H         PUBLIC        MINCS0L
  X:F021H         PUBLIC        MAXCS0L
BL51 BANKED LINKER/LOCATER V6.22                                                      05/19/2022  10:32:59  PAGE 5


  X:F002H         PUBLIC        PW1YH
  D:00D0H         PUBLIC        PSW
  X:F016H         PUBLIC        PW2YH
  X:F030H         PUBLIC        PW3YH
  D:00C0H         PUBLIC        IRCON
  -------         PROC          MAIN
  C:0341H         LINE#         47
  C:0341H         LINE#         48
  C:0341H         LINE#         49
  C:0344H         LINE#         50
  C:0346H         LINE#         60
  C:0354H         LINE#         61
  C:0362H         LINE#         62
  C:0370H         LINE#         64
  C:037BH         LINE#         66
  C:037BH         LINE#         67
  C:037BH         LINE#         68
  C:0380H         LINE#         69
  C:0380H         LINE#         70
  C:0382H         LINE#         71
  C:0384H         LINE#         73
  C:038EH         LINE#         74
  C:038EH         LINE#         75
  C:0390H         LINE#         76
  C:0392H         LINE#         78
  C:0395H         LINE#         79
  C:0398H         LINE#         80
  C:039BH         LINE#         81
  C:039EH         LINE#         82
  C:03A1H         LINE#         83
  C:03A4H         LINE#         84
  C:03A7H         LINE#         85
  C:03AAH         LINE#         87
  C:03B5H         LINE#         88
  C:03B5H         LINE#         89
  C:03B5H         LINE#         90
  -------         ENDPROC       MAIN
  -------         PROC          GPIO_INITIALIZATION
  C:0031H         LINE#         98
  C:0031H         LINE#         99
  C:0031H         LINE#         101
  C:0037H         LINE#         102
  C:003DH         LINE#         103
  C:0043H         LINE#         104
  C:0049H         LINE#         105
  -------         ENDPROC       GPIO_INITIALIZATION
  -------         ENDMOD        MAIN

  -------         MODULE        OPTIONS_SN8F5835
  C:7FF0H         PUBLIC        CRC_CHECK_DATA
  N:001EH         SYMBOL        BIT16_BYPASS1P_H
  N:00AFH         SYMBOL        BIT16_BYPASS1P_L
  N:0008H         SYMBOL        CK_FINE_TUNING_SET
  N:0018H         SYMBOL        CLOCKSRC_SET
  N:00C0H         SYMBOL        EXTERNAL_CLOCKRATE_SET
  N:00A0H         SYMBOL        IHRC32M_CLOCKRATE_SET
  N:0004H         SYMBOL        ISP_EN_SET
BL51 BANKED LINKER/LOCATER V6.22                                                      05/19/2022  10:32:59  PAGE 6


  N:0001H         SYMBOL        NOISEFILT_SET
  N:0030H         SYMBOL        RESETPIN_SET
  N:8000H         SYMBOL        ROM_SIZE
  N:0003H         SYMBOL        SECURITY_SET
  N:00C0H         SYMBOL        WATCHCLK_SET
  N:00A0H         SYMBOL        WATCHDOG_SET
  N:00C0H         SYMBOL        XTAL12M_CLOCKRATE_SET
  N:00E0H         SYMBOL        XTAL4M_CLOCKRATE_SET
  -------         ENDMOD        OPTIONS_SN8F5835

  -------         MODULE        UART0
  C:0000H         SYMBOL        _ICE_DUMMY_
  D:0080H         PUBLIC        P0
  D:0090H         PUBLIC        P1
  D:00B0H         PUBLIC        P3
  C:0056H         PUBLIC        UART0_ReceivedDone
  D:00C8H         PUBLIC        P4
  D:00A0H         PUBLIC        TTCON
  D:00A8H         PUBLIC        IEN0
  D:00B8H         PUBLIC        IEN1
  D:009BH         PUBLIC        S0CON2
  C:04B0H         PUBLIC        _UART0_TransmitData
  D:00D8H         PUBLIC        CSCON4
  D:009DH         PUBLIC        S0RELH
  D:0087H         PUBLIC        PCON
  D:009CH         PUBLIC        S0RELL
  D:0088H         PUBLIC        TCON
  B:0080H.6       PUBLIC        P06
  C:0066H         PUBLIC        ISR_UART0_RX
  D:00F9H         PUBLIC        P0M
  D:0099H         PUBLIC        S0BUF
  C:0216H         PUBLIC        _UART0_Init
  D:0098H         PUBLIC        S0CON
  D:0018H         PUBLIC        stUART0_Hardware
  B:00B8H.3       PUBLIC        EU0RX
  D:00D0H         PUBLIC        PSW
  D:00C0H         PUBLIC        IRCON
  -------         PROC          _UART0_INIT
  D:0007H         SYMBOL        bUartBaudRate
  D:0001H         SYMBOL        bRxBufAddress
  D:003AH         SYMBOL        bLength
  C:0216H         LINE#         59
  C:0216H         LINE#         60
  C:0216H         LINE#         61
  C:021BH         LINE#         62
  C:021EH         LINE#         65
  C:0221H         LINE#         66
  C:0224H         LINE#         69
  C:0227H         LINE#         71
  C:022AH         LINE#         72
  C:022AH         LINE#         74
  C:022DH         LINE#         75
  C:022FH         LINE#         77
  C:022FH         LINE#         79
  C:0232H         LINE#         80
  C:0235H         LINE#         81
  C:0238H         LINE#         83
BL51 BANKED LINKER/LOCATER V6.22                                                      05/19/2022  10:32:59  PAGE 7


  C:0266H         LINE#         84
  C:0266H         LINE#         85
  C:0269H         LINE#         87
  C:026BH         LINE#         89
  C:026BH         LINE#         90
  C:026BH         LINE#         92
  C:026DH         LINE#         94
  C:026DH         LINE#         95
  C:0270H         LINE#         96
  C:0272H         LINE#         98
  C:0272H         LINE#         99
  C:0275H         LINE#         100
  C:0277H         LINE#         102
  C:0277H         LINE#         103
  C:027AH         LINE#         104
  C:027CH         LINE#         106
  C:027CH         LINE#         107
  C:027CH         LINE#         108
  C:027CH         LINE#         110
  C:027FH         LINE#         112
  C:0281H         LINE#         114
  C:0281H         LINE#         115
  C:0284H         LINE#         116
  C:0284H         LINE#         118
  C:0284H         LINE#         119
  C:0284H         LINE#         120
  C:0284H         LINE#         121
  C:0284H         LINE#         124
  C:0288H         LINE#         125
  C:0288H         LINE#         126
  C:028BH         LINE#         127
  C:0291H         LINE#         128
  C:02A5H         LINE#         129
  C:02ACH         LINE#         130
  C:02ACH         LINE#         133
  C:02AFH         LINE#         134
  C:02B2H         LINE#         137
  C:02B4H         LINE#         138
  -------         ENDPROC       _UART0_INIT
  -------         PROC          _UART0_TRANSMITDATA
  D:0036H         SYMBOL        bptrData
  D:0005H         SYMBOL        bLength
  C:04B0H         LINE#         148
  C:04B6H         LINE#         149
  C:04B6H         LINE#         150
  C:04BCH         LINE#         151
  C:04BCH         LINE#         153
  C:04CFH         LINE#         154
  C:04D5H         LINE#         155
  C:04D8H         LINE#         156
  C:04DAH         LINE#         157
  -------         ENDPROC       _UART0_TRANSMITDATA
  -------         PROC          UART0_RECEIVEDDONE
  C:0056H         LINE#         164
  C:0056H         LINE#         165
  C:0056H         LINE#         166
  C:005BH         LINE#         167
BL51 BANKED LINKER/LOCATER V6.22                                                      05/19/2022  10:32:59  PAGE 8


  C:005BH         LINE#         168
  C:005EH         LINE#         169
  C:0060H         LINE#         170
  C:0060H         LINE#         172
  C:0060H         LINE#         173
  C:0061H         LINE#         174
  C:0061H         LINE#         175
  -------         ENDPROC       UART0_RECEIVEDDONE
  -------         PROC          ISR_UART0_RX
  C:0066H         LINE#         184
  C:0077H         LINE#         188
  C:008AH         LINE#         189
  C:009BH         LINE#         190
  C:009BH         LINE#         191
  C:00A4H         LINE#         192
  C:00A7H         LINE#         193
  C:00A7H         LINE#         195
  C:00AAH         LINE#         196
  -------         ENDPROC       ISR_UART0_RX
  -------         ENDMOD        UART0

  -------         MODULE        UART1
  C:0000H         SYMBOL        _ICE_DUMMY_
  D:0080H         PUBLIC        P0
  D:0090H         PUBLIC        P1
  D:00B0H         PUBLIC        P3
  D:00C8H         PUBLIC        P4
  C:051BH         PUBLIC        UART1_ReceivedDone
  D:00A0H         PUBLIC        TTCON
  D:00A8H         PUBLIC        IEN0
  D:00B8H         PUBLIC        IEN1
  D:009BH         PUBLIC        S0CON2
  C:0003H         PUBLIC        _UART1_TransmitData
  D:00D8H         PUBLIC        CSCON4
  D:00C4H         PUBLIC        S1RELH
  D:0087H         PUBLIC        PCON
  B:0090H.1       PUBLIC        P11
  D:00C3H         PUBLIC        S1RELL
  D:0088H         PUBLIC        TCON
  C:03B7H         PUBLIC        ISR_UART1_RX
  D:00FAH         PUBLIC        P1M
  D:0099H         PUBLIC        S0BUF
  D:00C2H         PUBLIC        S1BUF
  D:0098H         PUBLIC        S0CON
  C:0173H         PUBLIC        _UART1_Init
  D:00C1H         PUBLIC        S1CON
  D:0022H         PUBLIC        stUART1_Hardware
  D:00D0H         PUBLIC        PSW
  D:00C0H         PUBLIC        IRCON
  -------         PROC          _UART1_INIT
  D:0007H         SYMBOL        bUartBaudRate
  D:0001H         SYMBOL        bRxBufAddress
  D:003AH         SYMBOL        bLength
  C:0173H         LINE#         56
  C:0173H         LINE#         57
  C:0173H         LINE#         58
  C:0178H         LINE#         59
BL51 BANKED LINKER/LOCATER V6.22                                                      05/19/2022  10:32:59  PAGE 9


  C:017BH         LINE#         61
  C:017EH         LINE#         62
  C:0181H         LINE#         65
  C:0184H         LINE#         67
  C:0187H         LINE#         68
  C:0187H         LINE#         70
  C:018AH         LINE#         71
  C:018CH         LINE#         73
  C:018CH         LINE#         75
  C:018FH         LINE#         76
  C:0192H         LINE#         77
  C:0195H         LINE#         79
  C:01C3H         LINE#         80
  C:01C3H         LINE#         81
  C:01C6H         LINE#         82
  C:01C6H         LINE#         83
  C:01C8H         LINE#         85
  C:01C8H         LINE#         86
  C:01CBH         LINE#         87
  C:01CEH         LINE#         88
  C:01D0H         LINE#         90
  C:01D0H         LINE#         91
  C:01D3H         LINE#         92
  C:01D5H         LINE#         94
  C:01D5H         LINE#         95
  C:01D8H         LINE#         96
  C:01DAH         LINE#         98
  C:01DAH         LINE#         99
  C:01DDH         LINE#         100
  C:01DFH         LINE#         102
  C:01DFH         LINE#         103
  C:01DFH         LINE#         104
  C:01DFH         LINE#         106
  C:01E2H         LINE#         108
  C:01E4H         LINE#         110
  C:01E4H         LINE#         111
  C:01E7H         LINE#         112
  C:01E7H         LINE#         114
  C:01E7H         LINE#         115
  C:01E7H         LINE#         116
  C:01E7H         LINE#         117
  C:01E7H         LINE#         120
  C:01EBH         LINE#         121
  C:01EBH         LINE#         122
  C:01EEH         LINE#         123
  C:01F4H         LINE#         124
  C:0208H         LINE#         125
  C:020FH         LINE#         126
  C:020FH         LINE#         129
  C:0212H         LINE#         130
  C:0215H         LINE#         131
  -------         ENDPROC       _UART1_INIT
  -------         PROC          _UART1_TRANSMITDATA
  D:003BH         SYMBOL        bptrData
  D:0005H         SYMBOL        bLength
  C:0003H         LINE#         142
  C:0009H         LINE#         143
BL51 BANKED LINKER/LOCATER V6.22                                                      05/19/2022  10:32:59  PAGE 10


  C:0009H         LINE#         144
  C:000FH         LINE#         145
  C:000FH         LINE#         147
  C:0022H         LINE#         148
  C:0028H         LINE#         149
  C:002BH         LINE#         150
  C:002DH         LINE#         151
  C:0030H         LINE#         152
  -------         ENDPROC       _UART1_TRANSMITDATA
  -------         PROC          UART1_RECEIVEDDONE
  C:051BH         LINE#         159
  C:051BH         LINE#         160
  C:051BH         LINE#         161
  C:0520H         LINE#         162
  C:0520H         LINE#         163
  C:0523H         LINE#         164
  C:0525H         LINE#         165
  C:0525H         LINE#         167
  C:0525H         LINE#         168
  C:0526H         LINE#         169
  C:0526H         LINE#         170
  -------         ENDPROC       UART1_RECEIVEDDONE
  -------         PROC          ISR_UART1_RX
  C:03B7H         LINE#         178
  C:03C8H         LINE#         180
  C:03DBH         LINE#         181
  C:03ECH         LINE#         182
  C:03ECH         LINE#         183
  C:03F5H         LINE#         184
  C:03F8H         LINE#         185
  C:03F8H         LINE#         187
  C:03FBH         LINE#         188
  -------         ENDPROC       ISR_UART1_RX
  -------         ENDMOD        UART1

  -------         MODULE        UART2
  C:0000H         SYMBOL        _ICE_DUMMY_
  D:0080H         PUBLIC        P0
  D:0090H         PUBLIC        P1
  D:00B0H         PUBLIC        P3
  D:00C8H         PUBLIC        P4
  C:0527H         PUBLIC        UART2_ReceivedDone
  D:00A0H         PUBLIC        TTCON
  D:00A8H         PUBLIC        IEN0
  D:00B8H         PUBLIC        IEN1
  D:009BH         PUBLIC        S0CON2
  C:040AH         PUBLIC        _UART2_TransmitData
  D:00CFH         PUBLIC        DEGCMD
  D:00D8H         PUBLIC        CSCON4
  D:0087H         PUBLIC        PCON
  D:00CCH         PUBLIC        S2RELH
  B:00C8H.0       PUBLIC        P40
  D:0088H         PUBLIC        TCON
  D:00CBH         PUBLIC        S2RELL
  C:045DH         PUBLIC        ISR_UART2_RX
  D:00FCH         PUBLIC        P4M
  D:00CAH         PUBLIC        S2BUF
BL51 BANKED LINKER/LOCATER V6.22                                                      05/19/2022  10:32:59  PAGE 11


  D:0098H         PUBLIC        S0CON
  C:00C6H         PUBLIC        _UART2_Init
  D:00C9H         PUBLIC        S2CON
  D:002CH         PUBLIC        stUART2_Hardware
  B:00B8H.7       PUBLIC        EU2RX
  D:00D0H         PUBLIC        PSW
  D:00C0H         PUBLIC        IRCON
  -------         PROC          _UART2_INIT
  D:0007H         SYMBOL        bUartBaudRate
  D:0001H         SYMBOL        bRxBufAddress
  D:003AH         SYMBOL        bLength
  C:00C6H         LINE#         58
  C:00C6H         LINE#         59
  C:00C6H         LINE#         61
  C:00C9H         LINE#         62
  C:00D3H         LINE#         65
  C:00D6H         LINE#         66
  C:00D9H         LINE#         69
  C:00DCH         LINE#         72
  C:00DFH         LINE#         74
  C:00E2H         LINE#         75
  C:00E2H         LINE#         77
  C:00E5H         LINE#         78
  C:00E7H         LINE#         80
  C:00E7H         LINE#         82
  C:00EAH         LINE#         83
  C:00EDH         LINE#         84
  C:00F0H         LINE#         86
  C:011EH         LINE#         87
  C:011EH         LINE#         88
  C:0121H         LINE#         89
  C:0121H         LINE#         90
  C:0123H         LINE#         92
  C:0123H         LINE#         93
  C:0126H         LINE#         94
  C:0129H         LINE#         95
  C:012BH         LINE#         97
  C:012BH         LINE#         98
  C:012EH         LINE#         99
  C:0130H         LINE#         101
  C:0130H         LINE#         102
  C:0133H         LINE#         103
  C:0135H         LINE#         105
  C:0135H         LINE#         106
  C:0138H         LINE#         107
  C:013AH         LINE#         109
  C:013AH         LINE#         110
  C:013AH         LINE#         111
  C:013AH         LINE#         113
  C:013DH         LINE#         115
  C:013FH         LINE#         117
  C:013FH         LINE#         118
  C:0142H         LINE#         119
  C:0142H         LINE#         121
  C:0142H         LINE#         122
  C:0142H         LINE#         123
  C:0142H         LINE#         124
BL51 BANKED LINKER/LOCATER V6.22                                                      05/19/2022  10:32:59  PAGE 12


  C:0142H         LINE#         127
  C:0146H         LINE#         128
  C:0146H         LINE#         129
  C:0149H         LINE#         130
  C:014FH         LINE#         131
  C:0163H         LINE#         132
  C:016AH         LINE#         133
  C:016AH         LINE#         136
  C:016DH         LINE#         137
  C:0170H         LINE#         139
  C:0172H         LINE#         140
  -------         ENDPROC       _UART2_INIT
  -------         PROC          _UART2_TRANSMITDATA
  D:0036H         SYMBOL        bptrData
  D:0005H         SYMBOL        bLength
  C:040AH         LINE#         151
  C:0410H         LINE#         152
  C:0410H         LINE#         154
  C:0413H         LINE#         155
  C:0416H         LINE#         156
  C:0419H         LINE#         157
  C:0425H         LINE#         159
  C:042BH         LINE#         160
  C:042BH         LINE#         162
  C:043EH         LINE#         163
  C:0444H         LINE#         164
  C:0447H         LINE#         165
  C:0449H         LINE#         167
  C:044CH         LINE#         168
  C:044FH         LINE#         169
  C:0452H         LINE#         170
  C:045CH         LINE#         172
  -------         ENDPROC       _UART2_TRANSMITDATA
  -------         PROC          UART2_RECEIVEDDONE
  C:0527H         LINE#         179
  C:0527H         LINE#         180
  C:0527H         LINE#         182
  C:052CH         LINE#         183
  C:052CH         LINE#         184
  C:052FH         LINE#         185
  C:0531H         LINE#         186
  C:0531H         LINE#         188
  C:0531H         LINE#         189
  C:0532H         LINE#         190
  C:0532H         LINE#         191
  -------         ENDPROC       UART2_RECEIVEDDONE
  -------         PROC          ISR_UART2_RX
  C:045DH         LINE#         199
  C:046EH         LINE#         202
  C:0481H         LINE#         203
  C:0492H         LINE#         204
  C:0492H         LINE#         205
  C:049BH         LINE#         206
  C:049EH         LINE#         208
  C:049EH         LINE#         210
  C:04A1H         LINE#         211
  -------         ENDPROC       ISR_UART2_RX
BL51 BANKED LINKER/LOCATER V6.22                                                      05/19/2022  10:32:59  PAGE 13


  -------         ENDMOD        UART2

  -------         MODULE        ?C?CLDPTR
  C:04DBH         PUBLIC        ?C?CLDPTR
  -------         ENDMOD        ?C?CLDPTR

  -------         MODULE        ?C?CSTPTR
  C:04F4H         PUBLIC        ?C?CSTPTR
  -------         ENDMOD        ?C?CSTPTR

*** WARNING L16: UNCALLED SEGMENT, IGNORED FOR OVERLAY PROCESS
    SEGMENT: ?PR?UART0_RECEIVEDDONE?UART0

*** WARNING L16: UNCALLED SEGMENT, IGNORED FOR OVERLAY PROCESS
    SEGMENT: ?PR?_UART1_TRANSMITDATA?UART1

*** WARNING L16: UNCALLED SEGMENT, IGNORED FOR OVERLAY PROCESS
    SEGMENT: ?PR?UART2_RECEIVEDDONE?UART2

Program Size: data=63.0 xdata=50 code=1323
LINK/LOCATE RUN COMPLETE.  3 WARNING(S),  0 ERROR(S)
